:020000040800F2
:1000000000070020F1010008212C0008D92B00086E
:10001000012C0008D92B0008F92B0008F301000877
:10002000F3010008F3010008F3010008BD3C0008DB
:10003000F3010008F3010008F3010008F3010008D0
:10004000F3010008F3010008F3010008F3010008C0
:10005000F3010008F301000885500008AD500008C6
:10006000D5500008FD50000825510008F301000894
:10007000F3010008F3010008F3010008F301000890
:10008000F3010008F3010008F30100088D2B0008BC
:10009000B92B0008C92B0008F30100084D510008D6
:1000A000F3010008F3010008F3010008F301000860
:1000B000F3010008F3010008F3010008F301000850
:1000C000F3010008F3010008F3010008F301000840
:1000D000F30100082152000835520008F30100081E
:1000E000B1510008F3010008F3010008F301000812
:1000F000F3010008F3010008F3010008F301000810
:10010000F3010008F301000849520008F301000858
:10011000F3010008F3010008F3010008F3010008EF
:10012000F3010008F3010008F3010008F3010008DF
:10013000F3010008F3010008F3010008F3010008CF
:10014000F3010008F3010008F3010008F3010008BF
:10015000F3010008F3010008F3010008F3010008AF
:10016000F3010008F3010008F3010008F30100089F
:10017000F3010008F3010008F3010008F30100088F
:10018000F3010008F3010008F3010008F30100087F
:10019000F3010008F3010008F3010008F30100086F
:1001A000F3010008F3010008F3010008F30100085F
:1001B000F3010008F3010008F3010008F30100084F
:1001C000F3010008F3010008F3010008F30100083F
:1001D000F3010008F3010008F3010008F30100082F
:1001E0004D150008000000000000000000000000A5
:1001F00002E000F000F8FEE772B6374880F30888A6
:10020000364880F3098836483649086040F20000D5
:10021000CCF200004EF63471CEF200010860BFF35C
:100220004F8FBFF36F8F40F20000C0F2F0004EF628
:100230008851CEF200010860BFF34F8FBFF36F8F7C
:100240004FF00000E1EE100A4EF63C71CEF20001D4
:100250000860062080F31488BFF36F8F04F014FD4C
:1002600004F0ACFD4FF055301F491B4A91423CBF92
:1002700041F8040BFAE71D49184A91423CBF41F886
:10028000040BFAE71A491B4A1B4B9A423EBF51F82E
:10029000040B42F8040BF8E700201849184A914271
:1002A0003CBF41F8040BFAE704F0F2FC04F0D4FD83
:1002B000144C154DAC4203DA54F8041B8847F9E797
:1002C00000F042F8114C124DAC4203DA54F8041B12
:1002D0008847F9E704F0DABC00070020002300207B
:1002E0000000000808ED00E00001002000070020E9
:1002F00008560008002300208C23002090230020B3
:1003000078530020E0010008E4010008E40100083F
:10031000E40100082DE9F04F2DED108AC1F80CD052
:10032000C3689D46BDEC108ABDE8F08F002383F3BF
:1003300011882846A047002004F016F9FEE704F0D3
:100340009FF800DFFEE70000F8B501F07BF904F04C
:1003500035FC074604F084FC0546A8BB1F4B9F42B2
:1003600032D001339F4232D01D4B27F0FF029A4218
:1003700030D1F8B200F000FF2E4642F2107400F0C7
:1003800001FF08B10024264601F00EFD20B1032034
:1003900000F07AF80024264635B1124B9F4203D074
:1003A00004F056FC00242646002004F011FC0EB197
:1003B00000F080F801F066FA00F052FF204600F0ED
:1003C000CDF800F077F8F9E72E460024D7E7044689
:1003D0000126D4E7064641F28834D0E7010007B091
:1003E000000008B0263A09B008B501F0F7F8A0F10E
:1003F00020035842584108BD07B541F212030221BB
:1004000001A8ADF8043001F007F903B05DF804FB72
:1004100038B5302383F31188174803680BB104F013
:1004200061F9164A144800234FF47A7104F050F928
:10043000002383F31188124C236813B12368013B16
:100440002360636813B16368013B63600D4D2B78D3
:1004500033B963687BB9022001F0AAF932236360E3
:100460002B78032B07D163682BB9022001F0A0F988
:100470004FF47A73636038BD9023002011040008A4
:10048000B0240020A8230020084B187003280CD8A3
:10049000DFE800F008050208022001F087B9022019
:1004A00001F082B9024B00225A607047A823002055
:1004B000B024002010B501F077FC30B1204B0322AE
:1004C0001A70204B00225A6010BD1F4B1F4A1C4659
:1004D00019680131F8D004339342F9D162681C4B9A
:1004E0009A42F1D91B4B9B6803F1006303F58033FB
:1004F0009A42E9D204F080FB04F092FB002001F064
:10050000BBF80220FFF7C0FF134B1A6C00221A64DD
:10051000196E1A66196E596C5A64596E5A665B6E7A
:1005200072B64FF0E0233021C3F8084DD4E9003211
:1005300081F311889D4683F308881047C4E700BF04
:10054000A8230020B024002000000108200001089A
:10055000FFFF000800230020003802402DE9F04F83
:1005600093B0AC4B00902022FF210AA89D6801F0B7
:1005700033F9A94A1378A3B9A8480121036011707F
:10058000302383F3118803680BB104F0ABF8A44A5D
:10059000A24800234FF47A7104F09AF8002383F301
:1005A0001188009B13B19F4B009A1A609E4A009CD1
:1005B0001378032B1EBF002313709A4A4FF0000AD2
:1005C00018BF5360D3465646D146012001F0EEF8DD
:1005D00024B1944B1B68002B00F01582002000F022
:1005E000FDFF0390039B002B01DA00F081FE039BCB
:1005F000002BEDDB012001F0D7F8039B213B162BEC
:10060000E3D801A252F823F0650600088D06000821
:1006100021070008CB050008CB050008CB05000822
:10062000AB0700087B09000895080008F7080008D8
:100630001F09000845090008CB05000857090008F4
:10064000CB050008C909000805070008CB0500080C
:100650000D0A00087106000805070008CB05000810
:10066000F70800080220FFF7BFFE002840F0F581E0
:10067000009B0221BAF1000F08BF1C4605A841F2F9
:100680001233ADF8143000F0C7FF9EE74FF47A70D4
:1006900000F0A4FF071EEBDB0220FFF7A5FE0028F9
:1006A000E6D0013F052F00F2DA81DFE807F0030A08
:1006B0000D10133605230593042105A800F0ACFFA7
:1006C00017E054480421F9E758480421F6E7584850
:1006D0000421F3E74FF01C08404600F0CFFF08F17B
:1006E00004080590042105A800F096FFB8F12C0F2E
:1006F000F2D1012000FA07F747EA0B0B5FFA8BFBF8
:100700004FF0000901F0B4F826B10BF00B030B2BEE
:1007100008BF0024FFF770FE57E746480421CDE7E5
:10072000002EA5D00BF00B030B2BA1D10220FFF75D
:100730005BFE074600289BD0012000F09DFF0220B1
:10074000FFF7A2FE00261FFA86F8404600F0A4FF3D
:10075000044690B10021404600F0B6FF0136002863
:10076000F1D1BA46044641F21213022105A8ADF8B0
:1007700014303E4600F050FF27E70120FFF784FECB
:100780002546244B9B68AB4207D9284600F076FFEC
:10079000013040F067810435F3E7234B00251D70DD
:1007A000204BBA465D603E46ACE7002E3FF460AF9A
:1007B0000BF00B030B2B7FF45BAF0220FFF764FE03
:1007C000322000F00BFFB0F10008FFF651AF18F037
:1007D00003077FF44DAF0F4A926808EB050393427D
:1007E0003FF646AFB8F5807F3FF742AF124B01931B
:1007F000B84523DD4FF47A7000F0F0FE0390039AC1
:10080000002AFFF635AF019B039A03F8012B01374D
:10081000EDE700BF00230020AC240020902300203F
:1008200011040008B0240020A82300200423002085
:10083000082300200C230020AC230020C820FFF751
:10084000D3FD074600283FF413AF1F2D11D8C5F183
:10085000200242450AAB25F0030028BF42468349E7
:100860000192184400F0A6FF019A8048FF2100F091
:10087000B3FF4FEAA8037D490193C8F387022846D6
:1008800000F0B2FF064600283FF46DAF019B05EB78
:10089000830537E70220FFF7A7FD00283FF4E8AE05
:1008A00000F032FF00283FF4E3AE0027B846704B5B
:1008B0009B68BB4218D91F2F11D80A9B01330ED059
:1008C00027F0030312AA134453F8203C0593404633
:1008D000042205A901F020FA04378046E7E73846EC
:1008E00000F0CCFE0590F2E7CDF81480042105A8B5
:1008F00000F092FE06E70023642104A8049300F0B0
:1009000081FE00287FF4B4AE0220FFF76DFD0028C1
:100910003FF4AEAE049800F0DFFE0590E6E700235A
:10092000642104A8049300F06DFE00287FF4A0AEBB
:100930000220FFF759FD00283FF49AAE049800F01A
:10094000DBFEEAE70220FFF74FFD00283FF490AE00
:1009500000F0EAFEE1E70220FFF746FD00283FF441
:1009600087AE05A9142000F0E5FE04210746049097
:1009700004A800F051FE3946B9E7322000F02EFEFF
:10098000071EFFF675AEBB077FF472AE384A926859
:1009900007EB090393423FF66BAE0220FFF724FDFD
:1009A00000283FF465AE27F003074F44B9453FF4F4
:1009B000A9AE484600F062FE0421059005A800F0AB
:1009C0002BFE09F10409F1E74FF47A70FFF70CFDF3
:1009D00000283FF44DAE00F097FE002844D00A9B5B
:1009E00001330BD008220AA9002000F0FDFE0028E8
:1009F0003AD02022FF210AA800F0EEFEFFF7FCFC0F
:100A00001C4803F0B7FD13B0BDE8F08F002E3FF493
:100A10002FAE0BF00B030B2B7FF42AAE00236421C7
:100A200005A8059300F0EEFD074600287FF420AEF0
:100A30000220FFF7D9FC804600283FF419AEFFF7EB
:100A4000DBFC41F2883003F095FD059800F02EFFA5
:100A5000464600F00DFF3C46B7E5064652E64FF02D
:100A6000000905E6BA467EE637467CE6AC23002060
:100A700000230020A0860100094A136849F269009A
:100A800099B21B0C00FB01331360064B186844F24B
:100A9000506182B2000C01FB0200186080B2704706
:100AA000182300201423002010B500211022044632
:100AB00000F092FE034B03CB206061601868A060D9
:100AC00010BD00BF107AFF1FF0B5ADF54F7D6CACC7
:100AD0004FF4C47207460D462046002100F07CFE0C
:100AE00002F0A6F8244B4FF47A72B0FBF2F01860D3
:100AF00093E80700022384E807000DF5E9702382DC
:100B0000FFF7D2FF4FF4A6431C49238406A804F044
:100B100041FC192384F832310DF2E32206AB0DF1CA
:100B2000300C1E4603CE664510605160334602F11C
:100B30000802F6D1337813700DAE314601222046FB
:100B400000F0CEFE00230393AB7E029305F1190360
:100B5000019380B20123CDE904600093E97E04A3F0
:100B6000D3E90023384602F079FC0DF54F7DF0BD46
:100B70009E6AC421818A46EEB8240020A45300084E
:100B80002DE9F0412C4C237ADAB080460D465BBB50
:100B900027A9284600F0CAFF0746002842D19DF841
:100BA0009D60C82E3ED801464FF4A662204600F054
:100BB00013FE4FF48073C4F8F8314FF40073C4F897
:100BC0000C334FF44073C4F8203432460DF19E01CB
:100BD00004F1090000F0EEFD26449DF89C30777288
:100BE00023720BB9EB7E23728122002106AC27A869
:100BF00000F0F2FD0122214627A800F0DDFF0023CE
:100C00000393AB7E029305F1190380B2019328236D
:100C1000CDE904400093E97E05A3D3E900234046D3
:100C200002F01CFC5AB0BDE8F08100BFAFF30080B9
:100C300026417272DF25D7B700350020F0B5254E6A
:100C40004FF48A7505FB0065F1B096F8D83085F849
:100C5000DC300024D822214685F8E8403AA800F08C
:100C6000BBFD06F1090000F0AFFDD5F8E4308DF8CA
:100C7000F000C2B206AF06F109010DF1F100CDE9B5
:100C80003A3400F097FD394601223AA800F0CAFF35
:100C900080B2CDE9047008230127CDE9023706F1BF
:100CA000D803019330230093317A0B4807A3D3E98B
:100CB000002302F0D3FBA04206DD01F0B9FFC5F826
:100CC000E000384671B0F0BD2046FBE778F6339F70
:100CD00093CACD8D00350020D03400202DE9F0419D
:100CE0001D4D1E4E1E4F86B0284602F0E3FB034604
:100CF00058B30024CDE90344ADF81440027B8DF8CD
:100D0000142099684068029403AA03C21B68DFF8A4
:100D1000548043F00043029301F08CFF821941F1AB
:100D20000003009402A9384601F020FAA04205DD34
:100D3000284602F0C3FB88F80040D5E798F8003059
:100D4000072B05D8013388F8003006B0BDE8F081E4
:100D5000014802F0B3FBF8E7D034002040420F0016
:100D6000383A0020353A002070B50D4614461E462C
:100D700002F0D0FA50B9022E10D1012C0ED112A3DC
:100D8000D3E90023C5E90023012007E0282C10D077
:100D900005D8012C09D0052C0FD0002070BD302CB7
:100DA000FBD10BA3D3E90023ECE70BA3D3E900238A
:100DB000E8E70BA3D3E90023E4E70BA3D3E900237F
:100DC000E0E700BFAFF30080401DA12026812A0B81
:100DD00078F6339F93CACD8D9E6AC421818A46EEF0
:100DE00026417272DF25D7B7F017304A39059E5673
:100DF00038B505460E4C0021013500F065FCA4F81D
:100E00002C55B4F82C0500F047FC78B1B4F82C054B
:100E100000F052FC014648B9B4F82C0500F054FC2F
:100E2000B4F82C350133A4F82C35EAE738BD00BFFF
:100E30000035002010B50A4B0A4A1A6003F58053AA
:100E400093F870203AB9DC6E2CB1204601F024F8FA
:100E5000204601F061F9BDE81040034801F01CB8DC
:100E6000383A00205C540008904A00202DE9F04FE9
:100E70008FB000AF05460C4602F04CFA00284BD16B
:100E8000237E022B1BD1E38A012B18D101F0D0FE67
:100E90000646FFF7F1FD03464FF4C870DFF8D48231
:100EA000B3FBF0F206F5167602FB103316FA83F365
:100EB000C8F80030E37E33B9A74B00221A703C37E4
:100EC000BD46BDE8F08F07F12401204600F0E2FDA9
:100ED0000028F4D107F11400FFF7E6FD97F826404B
:100EE00007F11401224607F1270004F021FA002837
:100EF000E2D10F2C08D8984B1C70D8F80030A3F51D
:100F00001673C8F80030DAE797F824100029D6D015
:100F1000284602F0F7F9D2E7E38A282B33D010D81D
:100F2000012B2BD0052BCAD1BFF34F8F8B498C4B94
:100F3000CA6802F4E0621343CB60BFF34F8F00BF77
:100F4000FDE7302BBBD1874EE17E327A9142B6D19C
:100F5000607E3146002291F8DC50854200F0AD8081
:100F60000132042A01F58A71F5D1326840F6B831B0
:100F7000FA328A4294BF32603160A0E721462846A7
:100F8000FFF7A2FD9BE721462846FFF7F9FD96E70C
:100F9000B2F8EC507B6005F103094FEA99094FEA7A
:100FA0008902D11DC908A8EBC1039D46EB4600216B
:100FB000584600F011FC04F1EE012A46314458462F
:100FC00000F0F8FB7B6813B9012000F055FB96F8A0
:100FD000D20000F061FB044630B9307200F094FB9F
:100FE000204600F049FBB0E0D6F8D4203AB996F894
:100FF000D200B6F82C25824201D8FFF7F9FED6F8C8
:10100000D4202A44944208D296F8D200B6F82C256F
:101010000130824201D8FFF7EBFE70685FFA89F277
:10102000594600F0E1FB08B9C54679E0726896F8C8
:10103000D2002A447260D6F8D42005EB0209C6F823
:10104000D49000F029FB814509D396F8D220D6F838
:10105000D4000132001B86F8D220C6F8D400FF2D40
:101060000FD80024347200F04FFB204600F004FB40
:1010700000F09AFE3C4B188108B9FFF71BFAC546F1
:101080001DE7BB6896F8D9000AFB0362FB68D2F83B
:10109000E41082F8E83001F58061C2F8E030C2F86F
:1010A000E410FFF7CBFDFFF719FE96F8D9200132C7
:1010B00002F0030286F8D920B6E74FF48A7A0AFBD9
:1010C00002F505F1EA013144204600F0DFFDF86049
:1010D00000287FF4F4AE3544012285F8E82001F0C1
:1010E000A7FDD5F8E020D6ED007ADFED206A801A62
:1010F000192838BF192040F6B832904228BF104650
:10110000B8EE677A07EE900AF8EEE77A67EEA67A0D
:10111000DFED176AE7EE267AFCEEE77AC6ED007A95
:1011200096F8D9307168BB600AFB03F4321992F863
:10113000E8505DB1D2F8E4308B42E8463FF428AF86
:10114000002182F8E810C2F8E010C5467368064A2C
:101150009B0A01331381B2E6C934002000ED00E0A0
:101160000400FA0500350020B8240020CDCCCC3D89
:101170006666663FCC340020014B1870704700BF94
:10118000C424002030B54FF000542C4B22689A4202
:1011900085B023D1637D0BB3294A2A481370237D80
:1011A00003724FF48073C0F8F8314FF40073C0F845
:1011B0000C3300254FF44073C0F820342249C0F8A6
:1011C000E450C922093000F0F5FA2046E022294611
:1011D00000F002FB0124204605B030BD03F04AFDBB
:1011E000044608B90024F6E7184A194D136C43F079
:1011F00000731364AA6D174B9A42F3D12B6E013B17
:101200007E2BEFD8144A07CA01AB83E807001846C3
:10121000032100F097FD6B6D83424FF00003E1D195
:101220002A6D8A4201BFAB65054B2A6E1A7003BF57
:101230000A4BEA6D1A601C46CDE700BF9AAD44C563
:10124000C424002000350020160000200038024091
:10125000006600405041A0B05866004010230020B6
:1012600037B51A4D00F0A0FD02236B71184B288191
:1012700019681848012201F075FB00230193164BF1
:10128000164900931648174B4FF4805202F012F89B
:10129000154B197811B1124802F034F801F0C8FC6E
:1012A0000446FFF7E9FB4FF4C873B0FBF3F202FB0F
:1012B000130304F5167010FA83F00C4B186003F05A
:1012C000CFFC08B10F232B8103B030BDB824002020
:1012D00010230020383A0020690D0008C82400209F
:1012E000D03400206D0E0008C4240020CC3400202F
:1012F0002DE9F04F2DED028B8CA7D7E900670FF297
:101300003429D9E90089844C95B00DAD9FED808BCF
:10131000FFF7E4FCDFF824B200230C93ADF83C3077
:101320000D936B6000230DF125028DED008B4FF0C6
:10133000010A09A958468DF825308DF824A001F03E
:10134000BFFA9DF824200023002A40F0AE802046FA
:1013500001F0E0FF0546002847D1DFF8E4B101F0D5
:1013600067FCDBF8003098423FD301F061FC079046
:10137000FFF782FB079A4FF4C873B0FBF3F101FB50
:10138000130302F5167010FA83F0CBF80000DFF8B3
:10139000B4B19BF800100791002914BF2B465346A7
:1013A00010A88DF83030FFF77FFB0799C1F11002CC
:1013B000D2B2062A10AB28BF062219440DF1310023
:1013C000079200F0F7F9079A0CAB039318230293E6
:1013D0000132524BD2B2CDE900A304923B463246D1
:1013E000204601F0DDFF8BF8005001F021FC4C4A53
:1013F0004C4D1368C31AB3F57A7F32D3106001F0F5
:1014000019FC02460B46204602F062F8204601F025
:1014100081FF30B32B7ADFF830A1002B14BF0323F8
:1014200002238AF8053001F003FC0DF1400B4FF464
:101430007A730122B0FBF3F05946CAF80000504617
:1014400000F000FB18230293374B019380B240F267
:101450005513CDE903B0009342464B46204601F0B8
:101460009FFF2B7AABB101F0E3FB4FF0000A8346FC
:101470004FF48A7295F8D900504400F0030002FB43
:10148000005393F8E81071B30AF1010ABAF1040F9E
:10149000F0D1C82003F06EF82B7A002B7FF435AF23
:1014A00015B0BDEC028BBDE8F08F1946102210A8D4
:1014B00000F092F90DF126030AAA0CA9584600F093
:1014C0005BFF95E8030011AB83E803009DF83C3017
:1014D0008DF84C300C9B109310A9DDE90A232046AF
:1014E00002F0CAF91EE7D3F8E01049B12B68FA2BD5
:1014F00038BFFA23ABEB01010533B1EB430FC3D384
:10150000FFF79CFB4FF48A720028BDD1C1E700BFF2
:101510000000000000000000D0340020C83400208B
:10152000303A002000350020343A0020401DA12030
:1015300026812A0BF1C6A7C1D068080F383A0020CF
:10154000CC340020C9340020B824002008B5054858
:1015500000F0B0FFBDE80840034A0449002003F052
:10156000C3BE00BF383A00206C4B0020350E000887
:101570002DE9F84F4FF47A73DFF85880DFF8589070
:1015800006460D4602FB03F7002498F900305A1C6A
:101590005FFA84FA01D0A34212D159F824000368FB
:1015A0002A46D3F820B031463B46D847854207D17A
:1015B000074B012083F800A0BDE8F88F0124E4E781
:1015C000002CFBD04FF4FA7002F0D4FF0020F3E7B8
:1015D000604B00201C2300202023002007B500239F
:1015E000024601210DF107008DF80730FFF7C0FF1B
:1015F00020B19DF8070003B05DF804FB4FF0FF3009
:10160000F9E700000A4608B50421FFF7B1FF80F0B2
:101610000100C0B2404208BD30B4074B0A461978F9
:10162000064B53F821402368DD69054B0146AC4663
:10163000204630BC604700BF604B002020230020C4
:10164000A086010070B503F069F9094E094D30809C
:10165000002428683388834208D903F059F92B689D
:1016600004440133B4F5803F2B60F2D370BD00BF5A
:10167000624B0020204B002003F0FEB900F1006017
:1016800000F580300068704700F10060920000F5BE
:10169000803003F089B90000054B1A68054B1B88A0
:1016A0009B1A834202D9104403F032B900207047DC
:1016B000204B0020624B0020024B1B68184403F0B3
:1016C0002FB900BF204B0020024B1B68184403F0C9
:1016D0003FB900BF204B002010F003030AD1B0F542
:1016E000047F05D200F10050A0F51040D0F800387A
:1016F000184670470023FBE700F10050A0F51040AA
:10170000D0F8100A70470000064991F8243033B130
:101710000023086A81F824300822FFF7B5BF0120B2
:10172000704700BF244B0020014B1868704700BF72
:10173000002004E070B5194B1D68194B0138C5F342
:101740000B0408442D0C04221E88A6420BD15C68B1
:101750000A46013C824213460FD214F9016F4EB182
:1017600002F8016BF6E7013A03F10803ECD181427C
:101770000B4602D22C2203F8012B0A4A05241688B4
:10178000AE4204D1984284BF967803F8016B013CC5
:1017900002F10402F3D1581A70BD00BF002004E02A
:1017A00000540008EC530008704700007047000028
:1017B0007047000010B50023934203D0CC5CC454A2
:1017C0000133F9E710BD000003460246D01A12F9B2
:1017D000011B0029FAD1704702440346934202D00C
:1017E00003F8011BFAE770472DE9F8431F4D144633
:1017F00095F824200746884652BBDFF870909CB3CA
:1018000095F824302BB92022FF2148462F62FFF79C
:10181000E3FF95F82400C0F10802A24228BF224647
:10182000D6B24146920005EB8000FFF7C3FF95F862
:101830002430A41B1E44F6B2082E17449044E4B290
:1018400085F82460DBD1FFF75FFF0028D7D108E0DF
:101850002B6A03EB82038342CFD0FFF755FF0028AA
:10186000CBD10020BDE8F8830120FBE7244B00200A
:10187000024B1A78024B1A70704700BF604B002071
:101880001C23002010B5074C074920684FF4E133B2
:101890000B6002F05BFD60680349BDE8104002F098
:1018A00055BD00BF202300204C4B0020094B10B534
:1018B0001422044600211846FFF78EFF064A074B04
:1018C000127804600146BDE8104053F8220002F08F
:1018D0003DBD00BF4C4B0020604B0020202300206A
:1018E0002DE9F3470D46044600219046284640F274
:1018F0007912FFF771FF234620220021284601F0CC
:101900005DFF231D02222021284601F057FF631DA1
:1019100003222221284601F051FFA31D0322252185
:10192000284601F04BFF04F1080310222821284625
:1019300001F044FF04F1100308223821284601F089
:101940003DFF04F1110308224021284601F036FF33
:1019500004F1120308224821284601F02FFF04F168
:10196000140320225021284601F028FF04F1180317
:1019700040227021284601F021FF04F120030822B3
:10198000B021284601F01AFF04F121030822B821F2
:10199000284601F013FF04F12207C0263B463146DA
:1019A00008222846083601F009FFB6F5A07F07F1A6
:1019B0000107F3D194F832308DF8073031460DF13C
:1019C00007030822284601F0F9FE002604F1330A35
:1019D0009DF807304FEAC6099E4209F5A47720D347
:1019E00094F83231502B28BF50238DF80730B8F1CE
:1019F000000F08D139460DF107030722284601F0F0
:101A0000DDFE09F24F17002604F233149DF807306B
:101A10009E4207EBC6010DD30731C80802B0BDE8EE
:101A2000F0870AEB060308223946284601F0C6FE75
:101A30000136CDE7A3190822284601F0BFFE013682
:101A4000E4E7000013B50446084600210160234680
:101A5000C0F803102022019001F0B0FE0198231D70
:101A60000222202101F0AAFE0198631D03222221F7
:101A700001F0A4FE0198A31D0322252101F09EFE82
:101A8000019804F108031022282101F097FE072095
:101A900002B010BDF7B5047F05460E462CB1838A0F
:101AA000122B02D9012003B0F0BD002319460722F2
:101AB0000096284601F046FD731C00930122002386
:101AC0000721284601F03EFDD4B9B31C009305223E
:101AD00023460821284601F035FD0D24B378102B4C
:101AE000E0D83746B278BB1B934210D32B7FA88A2D
:101AF0000734E408B3B9844294BF00200120D2E740
:101B0000AB8ADB00083BDB08B3700824E6E7FB1C6C
:101B10000093214600230822284601F013FD0834D3
:101B20000137DFE7201A18BF0120BCE7F7B5047FB3
:101B300005460E462CB1838ACA2B02D9012003B078
:101B4000F0BD0023194600960822284601F0FAFC51
:101B5000731CD4B90822009311462346284601F08D
:101B6000F1FC10247378C82BE8D8012372785F1C2D
:101B7000013B934210D32B7FA88A0734E408B3B902
:101B8000844294BF00200120D9E7AB8ADB00083BE8
:101B9000DB0873700824E5E7F3190093214600235E
:101BA0000822284601F0CEFC08343B46DEE7201A26
:101BB00018BF0120C3E70000F7B50D460446002119
:101BC000164628468122FFF707FE234608220021F9
:101BD000284601F0F3FD94F901206378002AB8BF8C
:101BE0007F238DF807309EB90DF1070307220821E6
:101BF000284601F0E3FD0F27002602349DF8073048
:101C00009E4207EBC60105D30731C80803B0F0BDFB
:101C10000827F1E7A3190822284601F0CFFD013675
:101C2000ECE70000F7B50E460546002114463046A5
:101C3000CE22FFF7D1FD2B4628220021304601F0AD
:101C4000BDFD2B7AC82B28BFC8238DF807308CB96F
:101C50000DF1070308222821304601F0AFFD3024A2
:101C60002F469DF807207B1B934205D3E01DC0083B
:101C700003B0F0BD2824F3E707F109032146082249
:101C8000304601F09BFD08340137EAE7F7B5047FE1
:101C900005460E4634B1838AB3F5827F02D901200E
:101CA00003B0F0BD0096012310220021284601F068
:101CB00049FCDCB9B31C00930922234610212846B5
:101CC00001F040FC19247388B3F5807FE7D83746CC
:101CD0007288BB1B934210D32B7FA88A0734E40879
:101CE000B3B9844294BF00200120D9E7AB8ADB005E
:101CF000103BDB0873801024E5E73B1D0093214671
:101D000000230822284601F01DFC08340137DFE7D4
:101D1000201A18BF0120C3E730B5094D0A4491428B
:101D20000DD011F8013B5840082340F30004013B5B
:101D30002C4013F0FF0384EA5000F6D1EFE730BDEA
:101D40002083B8EDF7B54FF0FF33DFF854C0DFF86C
:101D500054E000EB81011A4688421CD050F8044B35
:101D6000019401AF042417F8015B82EA056208259B
:101D7000DB18164605F1FF355241002EBCBF83EA41
:101D80000C0382EA0E0215F0FF05F1D1013C14F0BC
:101D9000FF04E8D1E0E7D843D14303B0F0BD00BF72
:101DA0009336EAA9EBE1F042F7B5354A106851687D
:101DB0006B4603C36A4633493348082303F0C8FA25
:101DC000044688BB0A25314A106851686B4603C334
:101DD0006A462F492C48082303F0BAFA0446002823
:101DE00045D00369B3F5702F41D8B0F86620532A67
:101DF0003DD1284A024402F15C018B4237D35C3B5F
:101E0000214900209E1AFFF787FF3246074604F15A
:101E100064010020FFF780FFA3689F4227D1E36899
:101E2000984208BF002522E00369B3F5702F25D83A
:101E3000428B532A20D1174A024402F110018B42EF
:101E400018D3103B104900209D1AFFF765FF2A4662
:101E5000064604F118010020FFF75EFFA3689E42CA
:101E600002D1E368984201D00D25ACE70025284651
:101E700003B0F0BD1025A6E70C25A4E70B25A2E7CB
:101E800020540008DCFF0E0000000108295400085F
:101E900090FF0E000800FFF710B5037C044613B94D
:101EA000006803F03DFA204610BD00000023BFF398
:101EB0005B8FC360BFF35B8FBFF35B8F8360BFF348
:101EC0005B8F7047BFF35B8F0068BFF35B8F70471A
:101ED00070B505460C30FFF7F5FF05F1080604461E
:101EE0003046FFF7EFFFA04206D930466D68FFF796
:101EF000E9FF2544281A70BD3046FFF7E3FF201A9A
:101F0000F9E7000070B50546406898B105F1080092
:101F1000FFF7D8FF05F10C0604463046FFF7D2FF65
:101F20008442304694BF6D680025FFF7CBFF013C2B
:101F30002C44201A70BD000038B50C460546FFF74A
:101F4000C7FFA04210D305F10800FFF7BBFF044410
:101F50006868B4FBF0F100FB1144BFF35B8F012014
:101F6000AC60BFF35B8F38BD0020FCE72DE9F0418A
:101F7000144607460D46FFF7C5FF844228BF0446B6
:101F8000D4B1B84658F80C6B4046FFF79BFF30447D
:101F9000286040467E68FFF795FF331A9C4203D8BD
:101FA0006C600120BDE8F0816B60A41B3B68AB60F6
:101FB0002044E8600220F5E72046F3E738B50C46F8
:101FC0000546FFF79FFFA04210D305F10C00FFF775
:101FD00079FF04446868B4FBF0F100FB1144BFF3DF
:101FE0005B8F0120EC60BFF35B8F38BD0020FCE706
:101FF0002DE9FF41884669460746FFF7B7FF6C4663
:1020000006B204EBC6060025B44209D06268206817
:1020100008EB0501FFF7CEFB636808341D44F3E7C6
:1020200029463846FFF7CAFF284604B0BDE8F081CC
:10203000F8B505460C300F46FFF744FF05F10806DA
:1020400004463046FFF73EFFA042304688BF6C682A
:10205000FFF738FF201A386020B130462C68FFF7B0
:1020600031FF2044F8BD000073B5144606460D4606
:10207000FFF72EFF844228BF04460190DCB101A97E
:102080003046FFF7D5FF019B33B93268C5E902330B
:10209000C5E9002401200CE09C4238BF019428606F
:1020A000019868608442F5D93368AB60241AEC600B
:1020B000022002B070BD2046FBE700002DE9FF4181
:1020C0000F466946FFF7D0FF6C4600B204EBC0052F
:1020D0000026AC4209D0D4F8048054F8081BB81983
:1020E0004246FFF767FB4644F3E7304604B0BDE8DD
:1020F000F081000038B50546FFF7E0FF04460146D1
:102100002846FFF719FF204638BD0000012188420C
:1021100038BF084603F0EEB808B103F001B97047C4
:1021200010B4026854681A4623465DF8044B1847F9
:102130000020704700207047704700000020704763
:102140000E20704700F5805090F8D800C0F3400092
:102150007047000000F5805090F9E00070470000E3
:1021600000F58050C0F8DC1001207047F7B50C680E
:10217000BDF8207014F0005473D10D7B082D70D879
:10218000302585F31188456AAE6876010CD4AC68B9
:10219000240108D4AC6814F0805460D184F3118811
:1021A000204603B0F0BD01240E6804F1180C002E87
:1021B000B8BFF6004FEA0C1CB4BF46F00406760523
:1021C00045F80C600E680FFA84FC16F0804F18BFBB
:1021D00005EB0C1E05EB0C1C1EBFDEF8806146F003
:1021E0000206CEF880610E7BCCF8846105EB041505
:1021F0008E68C5F88C614E68C5F88861DCF880513E
:1022000045F00105CCF8805141F2780500EB441C03
:10221000660105EB4414AC440444CCE900230D46AC
:10222000083401F10C0C55F804EB44F804EB654557
:10223000F9D12D882580841904F5805407F0030511
:1022400094F8946026F00B06354384F894500024EB
:1022500084F31188009700F035FD0120A1E70224E6
:10226000A2E74FF0FF309CE713B500F580540191D1
:10227000E06EFFF747FE1F280AD90199E06E202281
:10228000FFF7B6FEA0F120035842584102B010BD3E
:102290000020FBE708B5302383F3118800F5805058
:1022A000C06EFFF703FE002383F3118808BD000012
:1022B00000220260828142608260704710B5002275
:1022C0000023C0E900230023044603810C30FFF7FC
:1022D000EFFF204610BD0000F0B5054600F5805028
:1022E0000C4690F8D83013F0040FC3F3800108BFF8
:1022F000114661F3820380F8D83005EB441303F5EF
:102300008453103389B01B79D8074FEA44162FD570
:1023100082B319072ED46846FFF7D0FF05EB4413AC
:1023200003F5845303AA03F1080718685968144693
:1023300003C40833BB422246F7D1186820609B884B
:10234000A380DDE90E23CDE900230123ADF8083099
:102350002B6869461B6C28469847354405F584551B
:1023600010352B791A075CBF43F008032B7101E08D
:10237000002AF2D109B0F0BD2DE9F0479A4688B0A5
:10238000074688469146302383F3118807F5805429
:102390006846FFF793FFE06EFFF79AFD1F282AD9E2
:1023A000E06E20226946FFF7A5FE202823D103AD69
:1023B000444605AB2E4603CE9E4220606160354602
:1023C00004F10804F6D130682060B388A380DDE909
:1023D0000023C9E90023BDF80830AAF80030002323
:1023E00083F3118853464A464146384608B0BDE853
:1023F000F04700F02BBC002080F3118808B0BDE846
:10240000F08700002DE9F84F182204460F460430EB
:102410000021FFF7E1F92046234B40F8283BFFF766
:1024200047FF04F13800FFF749FF04F1580804F5AD
:1024300082554646183530462036FFF73FFFAE42FC
:10244000F9D104F580554FF480534FF00009C5E9E8
:102450001739C5F858800123EE6604F5875804F54E
:102460008456C5F8649085F8683085F87030183661
:1024700008F118084FF0000A4FF0000B46E908ABCE
:10248000A6F11800FFF714FF203646F8289C4645B1
:10249000F4D185F8E07017B1044800F0C3FB044B99
:1024A00063622046BDE8F88F5C540008345400088D
:1024B0000064004010B5044B197804464A1C1A7099
:1024C000FFF7A0FF204610BD684B00202DE9F04724
:1024D000002950D0294B2A4FB7FBF1F599428CBF08
:1024E0000A231123581EB5FBF3FC03FB1C53C4B293
:1024F0002BB102280346F5D80020BDE8F0870CF187
:10250000FF36B6F5806FF7D2C4EBC40E0EF10303AD
:102510004FEAE309C3F3C703A4EB030809F1010A77
:102520004FF47A755FFA88F009FB05555AFA88F876
:10253000B5FBF8F5B5F5617FC1BF0EF1FF33C3F30D
:10254000C703E01AC0B25C1C50FA84F40CFB04F41C
:10255000B7FBF4F4A142CFD1013BDBB20F2BCBD8B8
:102560000138C0B20728C7D80021107116809170B9
:10257000D3700120C1E70846BFE700BF3F420F000C
:1025800040787D0170B505460E464FF47A746B6A4B
:102590005B6803F00103B34207D04FF47A7001F097
:1025A000E9FF013CF3D1204670BD0120FCE70000AB
:1025B00070B5426A936913F0700F17D000230C4D69
:1025C000936141F2900400EB4312224411794E07CB
:1025D00009D5890707D5416A55F823608E601179BE
:1025E00041F0040111710133032BECD170BD00BF28
:1025F0004854000873B51D46436A16469A68D207C8
:10260000044609D59A6801219960C2F34002CDE9D8
:1026100000650021FFF760FE636A9A68D1050BD55B
:102620009A684FF480719960C2F34022CDE9006549
:1026300001212046FFF750FE636A9A68D2030BD54A
:102640009A684FF480319960C2F34042CDE9006549
:1026500002212046FFF740FE04F58053D3F8DC004A
:1026600010B103681B699847204602B0BDE870406E
:10267000FFF79EBFF8B50446466A002977D106F1F8
:102680000C073868800775D006EB01153868D5F857
:10269000B00110F0040FD5F8B0011ABFC00840F027
:1026A0000040400DA062D5F8B0C11CF0020F1CBF65
:1026B00040F08040A062D5F8B40106EB011100F0B3
:1026C0000F0084F83400D1F8B80184F82C00D1F858
:1026D000B801000A84F82D00D1F8B801000C84F884
:1026E0002E00D1F8B801000E84F82F00D1F8BC01FB
:1026F00084F83000D1F8BC01000A84F83100D1F828
:10270000BC01000C84F83200D1F8BC11090E84F829
:1027100033103821396004F1440004F1280104F138
:10272000340551F8046B40F8046BA942F9D10988CB
:102730000180C4E90E2321460023A4F8403051F85B
:10274000383B20461B6C984704F5805393F8D820FB
:10275000D3F8DC0042F0040283F8D82010B10368FB
:102760001B6998472046BDE8F840FFF721BF06F1F6
:10277000100786E7F8BD000010B5044600F05AFACD
:1027800002460B4652EA030102D0013A63F100030C
:102790000449086820B12146BDE81040FFF76ABF30
:1027A00010BD00BF644B0020F0B5302181F31188CB
:1027B000DFF848E000F583511831002441F2900C15
:1027C00000EB441565442E7977070ED4F6060CD538
:1027D000D1E9007697429E4107D2466A5EF824709E
:1027E000B7602E7946F004062E710134032C01F1F6
:1027F0002001E5D1002383F31188F0BD485400087F
:1028000008B5302383F31188FFF7D2FE002383F34A
:10281000118808BD2DE9F041436A0446986800F02C
:10282000E050B0F1E05F0E4622D0F8B1302383F3E0
:102830001188002504F5845741F2900804EB4513F4
:1028400043441B791A0706D50135032D07F12007EC
:10285000F4D1012007E05B07F6D43946304600F09A
:1028600083FA0028F0D1002383F31188BDE8F081BA
:102870000120FBE708B5302383F3118800F5805071
:10288000C06EFFF725FB002383F3118843090CBFBB
:102890000120002008BD0000F8B51D46002313707C
:1028A0000F4606461446FFF7E5FF80F0010038703A
:1028B00025B129463046FFF7ADFF2070F8BD000076
:1028C0002DE9B8410C4615461F46804600F0B2F986
:1028D0000B462178024609B9287850B14046FFF7E7
:1028E00063FFFFF78DFF3B462A462146FFF7D4FFE3
:1028F0000120BDE8B881000070B5302686F311884C
:10290000174B1A6C42F000721A641A6A42F0007295
:102910001A621A6A22F000721A62002383F3118885
:1029200000F5805494F8D83013F0010516D1A9B100
:1029300086F311880321132001F03CFB03211420AE
:1029400001F038FB0321152001F034FB94F8D83056
:1029500043F0010384F8D83085F3118870BD00BFBF
:10296000003802402DE9F04700F5805588B095F811
:10297000E030012B04468846164600F28280824FE2
:1029800057F823200AB947F82300D7F800A0C4F865
:102990001C8084F82060BAF1000F64D095F8E03014
:1029A000012B70D001212046FFF7A6FF302383F3CF
:1029B0001188626A136823F002031360626A136865
:1029C00043F001031360636A00275F6187F3118896
:1029D00001212046FFF7D6FD002800F09580E86E23
:1029E000FFF764FA04F58359BA4609F11809202261
:1029F00000216846FEF7F0FE02A8FFF759FCCDF86B
:102A000018A06A4609EB07030DF1180E9446BCE8BE
:102A10000300F44518605960624603F10803F5D1DC
:102A2000DCF80000186020379CF804201A71602F31
:102A3000DDD195F8D8306FF38203002785F8D830C0
:102A40006A4641462046ADF80070ADF802708DF838
:102A50000470FFF73BFD636A48BB4FF400421A6005
:102A600008B0BDE8F08741F2E800FFF74FFB814670
:102A700010B15146FFF7C6FCC7F80090B9F1000F3E
:102A80008CD10020ECE7386803681B6B984701463F
:102A9000002887D13868FFF72FFF3868036832466F
:102AA0005B684146984700287FF47CAFE9E76122E4
:102AB0001A609DF802309DF803201B06120402F4F0
:102AC000702203F040731343BDF80020C2F30902E3
:102AD00013439DF804201205022E02F4E0020CBFFD
:102AE0004FF0004100211343626A0B43D361636AD4
:102AF00013225A61626A136823F001031360394696
:102B00002046FFF73FFD08B9636AA6E795F8E03075
:102B100093BB616AD1F8002242F00102C1F80022A1
:102B2000616AD1F8002222F47C5222F00E02C1F830
:102B30000022616AD1F8002242F46062C1F80022EA
:102B4000626AC2F81432626AC2F80432626A41F6FA
:102B5000FF71C2F80C12626AC2F84032626AC2F8AF
:102B60004432636A0122C3F81C22626AD2F800323E
:102B700023F00103C2F8003295F8D83043F0020385
:102B800085F8D8306CE700BF644B002008B500F032
:102B900051F850EA0103024602D0421E61F10001E1
:102BA000044B186810B10B46FFF724FDBDE8084040
:102BB00001F0B8B8644B002008B50020FFF7DCFD39
:102BC000BDE8084001F0AEB808B50120FFF7D4FD1C
:102BD000BDE8084001F0A6B800B59BB0EFF309814D
:102BE00068226846FEF7E6FDEFF30583014B9B6B19
:102BF000FEE700BF00ED00E008B5FFF7EDFF0000C5
:102C000000B59BB0EFF3098168226846FEF7D2FD5C
:102C1000EFF30583014B5B6BFEE700BF00ED00E0C7
:102C2000FEE700000FB408B5029801F053FCFEE780
:102C300001F062BF01F044BF0139C9B202299EBF51
:102C400000EBC1000023C0E901337047F8B51B88D1
:102C50005B0705460E4615D4044600F11807BC4232
:102C600010D0636853B12B682846DB6B9847A36884
:102C7000C1B23246606898470834F0E7A368002B79
:102C8000F1D1F9E70120F8BD73B56C4684E8060080
:102C9000014600224E68D5B26EB98E685EB900EB6F
:102CA000C200021D94E80300013582E803001D7094
:102CB000012002B070BD0132032A01F10801E9D1FF
:102CC0000020F6E72DE9F04F89B00446BDF84870C2
:102CD0000E46054600F118084FF0000907F00407FA
:102CE0004FF0000A4FF0000BA84538D06B680BB9C5
:102CF000AB684BB157B923682046DB6B9847AB688C
:102D0000C1B23246686898470835EDE7B9F1000F5F
:102D1000FAD1CDE900ABADF80890334603AA06F12D
:102D2000080E186859689446ACE8030008337345E8
:102D30006246F6D11868CCF800009B88ACF80430E5
:102D4000FFF778FF0423ADF808302368CDE90001D0
:102D50001B6C6946204698474FF00109D4E70120D3
:102D600009B0BDE8F08F000030B503680968DD0FD9
:102D7000B5EBD17F23F0604421F060424FEAD1707F
:102D80000BD0002BB8BFA40C0029B8BF920C944202
:102D900002D034BF0120002030BD944205D1C1F3E0
:102DA0008070C3F380738342F6D194422CBF00201D
:102DB0000120F1E72DE9F041456A15B94162BDE80E
:102DC000F0814B6823F06047C3F38A464FEAD37E15
:102DD000C3F3807816EA230638BF3E46AC462B463E
:102DE0005A68BEEBD27F22F060440AD0002A18DA7B
:102DF000A40CB44217D19D420FD10D60DEE71346FB
:102E0000EEE7A74207D102F08044C2F38072424548
:102E10000BD054B1EFE708D2EDE7CCF800100B600F
:102E2000CDE7B44201D0B442E5D81A689C46002AE6
:102E3000E5D11960C3E700002DE9F047089D01F0D6
:102E400007044FEAD508224405F0070500EBD1003E
:102E50004FF47F49944201D1BDE8F08704F00707A1
:102E600005F0070A57453E4638BF5646C6F10806E4
:102E7000111B8E4228BF0E46E10808EBD50E415CBF
:102E800013F80EC0B94029FA06F721FA0AF1FFB289
:102E90008CEA010147FA0AF739408CEA010C03F881
:102EA0000EC034443544D5E780EA0120082341F2BE
:102EB000210201B24000002980B203F1FF33B8BF04
:102EC000504013F0FF03F4D17047000038B50C46B2
:102ED0008D18A54200D138BD14F8011BFFF7E4FF9F
:102EE000F7E7000042684AB113684360438981896B
:102EF00001339BB29942438138BF838110467047AA
:102F000070B588B0202204460D4668460021FEF7C1
:102F100063FC20460495FFF7E5FF024658B16B4677
:102F2000054608AE1C4603CCB442286069602346BF
:102F300005F10805F6D1104608B070BD082817D96C
:102F400009280CD00A280CD00B280CD00C280CD047
:102F50000D280CD00E2814BF4020302070470C20C4
:102F600070471020704714207047182070472020A9
:102F700070470000082817D90C280CD910280CD944
:102F800014280CD918280CD920280CD930288CBF2B
:102F90000F200E207047092070470A2070470B2031
:102FA00070470C2070470D20704700002DE9F84352
:102FB000078C072F04461ED9D0E9029800254FF64A
:102FC000FF73C5F12006A5F1200029FA05F108FAE2
:102FD00006F628FA00F031430143C9B21846FFF75C
:102FE00063FF0835402D0346EBD1E1693A46BDE861
:102FF000F843FFF76BBF4FF6FF70BDE8F8830000A2
:1030000010B54B6823B9CA8A63F30902CA8210BD9E
:1030100004691A681C600361C38A013BC3824A6069
:10302000EFE700002DE9F84F1D46CB8A0F46C3F3AA
:1030300009010529814692460B4630D00020AAB2EC
:1030400007F11A049EB2042E1FFA80F80FD890459B
:1030500003F1010306D3FB8A0A4462F30903FB82EE
:1030600001201AE01AF80060E6540130EAE79045C2
:10307000F1D2A1F1050B1C237C68BBFBF3F203FB2F
:1030800012BB1FFA8BF6002C45D14846FFF72AFFEA
:10309000044638B978606FF00200BDE8F88F4FF051
:1030A0000008E6E7002606607860ADB24FF0000B3E
:1030B000454510D90AEB0803221D13F8011B915551
:1030C000B1B208F101081B291FFA88F82BD0454539
:1030D00006F10106F1D8FB8AC3F30902154465F332
:1030E0000903BCE7013292B21C462368002BF9D1D8
:1030F0006B1F0B441C21B3FBF1F301339BB29A42CB
:10310000D3D2BBF1000FD0D14846FFF7EBFE20B978
:10311000C4F800B0BFE70122E7E7C0F800B05E46A0
:1031200020600446C1E74545D5D94846FFF7DAFE99
:1031300008B92060AFE7C0F800B000262060044660
:10314000B6E700002DE9F04F2DED028B1C4683B051
:103150005B69019207468846002B00F0A780238C0C
:103160002BB1E269002A00F0A180072B35D807F1C6
:103170000C00FFF7B7FE054638B96FF00205284688
:1031800003B0BDEC028BBDE8F08F14220021FEF7E6
:1031900023FB228CE16905F10800FEF70BFB208C74
:1031A000013080B2FFF7E6FEFFF7C8FE013880B2BB
:1031B0002084013028746369228C1B782A4403F030
:1031C0001F0363F03F0348F0004113723846696003
:1031D0002946FFF7EFFD0125D1E702339BB2072215
:1031E000C18A0633B3FBF2F3828A521A9BB292B2BF
:1031F0009342C2D800F10C034FF0000908EE103AD8
:103200004FF0800A4E464D4618EE100AFFF76AFE50
:1032100083460028B1D014220021FEF7DDFA002EEB
:103220003AD1019BABF8083002220BF1080E1FFACD
:1032300082FC0CF10100BCF1060F218C80B201D898
:103240008E422BD3FFF796FEFFF778FE6269127865
:10325000013802F01F028E4208BF4FF0400A42EAD6
:1032600049121BFA80F14AEA020A013048F0004292
:1032700081F808A08BF81000CBF804205946384696
:10328000FFF798FD238C0135B3422DB289F0010977
:103290004FF0000AB8D172E70022C6E7E169895D04
:1032A0000EF802100136B6B20132C0E76FF0010528
:1032B00065E70000F8B515460E46302200210446A9
:1032C0001F46FEF789FA069B6360B5F5001F079B52
:1032D000A76034BF6A094FF6FF72A36297B2E66136
:1032E00004F1100000239A4206D800230360A7824D
:1032F000E3822383E360F8BD066001333046203665
:10330000F1E7000003781BB94BB2002BC8BF017076
:103310007047000000787047F8B50C46C969074649
:1033200011B9238C002B37D1257E1F2D34D8387846
:1033300028BB228C072A2CD8268A36F003032BD1EF
:103340004FF6FF70FFF7C2FD20F00100310240048C
:1033500041EA0561400C41EA40254FF6FF722346E1
:1033600029463846FFF7EEFE002807DD626913782C
:103370000133DBB21F2B88BF00231370F8BD218AF5
:103380002D0645EA012505432046FFF70FFE0246BC
:10339000E5E76FF00300F1E76FF00100EEE70000F2
:1033A00070B58AB0044616460021282268461D469C
:1033B000FEF712FABDF83830ADF810300F9B0593C8
:1033C0009DF840308DF81830119B07936946BDF881
:1033D0004830ADF820302046CDE90265FFF79CFF6C
:1033E0000AB070BD2DE9F041D36905460C4616467A
:1033F0000BB9138C5BBB377E1F2F28D895F8008044
:10340000B8F1000F26D03046FFF7D0FD3378210207
:1034100041EAC33141EA0801338A41EA076141EADE
:1034200003410246334641F080012846FFF78AFEF9
:1034300000280ADD3378012B07D172691378013334
:10344000DBB21F2B88BF00231370BDE8F0816FF043
:103450000100FAE76FF00300F7E70000F0B58BB06A
:1034600004460D4617460021282268461E46FEF7F0
:10347000B3F99DF84C305A1E534253418DF8003039
:103480009DF84030ADF81030119B05939DF8483001
:103490008DF81830149B07936A46BDF85430ADF888
:1034A000203029462046CDE90276FFF79BFF0BB07E
:1034B000F0BD0000406A00B104307047436A1A68EA
:1034C000426202691A600361C38A013BC38270478A
:1034D0002DE9F041D0F82080194E14461D46414692
:1034E000002709B9BDE8F081D1E90223A21A65EBF2
:1034F0000303964277EB03031ED2036A8B420DD17E
:10350000FFF77EFD036A1B68036203690B60C38AD1
:103510000161016A013BC3828846E2E7FFF770FD63
:103520000B68C8F8003003690B60C38A0161013B76
:10353000C382D8F80010D4E788460968D1E700BFF5
:1035400080841E002DE9F04F8BB00D46DDF85090C1
:1035500014469B468046002800F01981B9F1000FFF
:1035600000F01581531E3F2B00F21181012A03D177
:10357000BBF1000F40F00B810023CDE90833B8F810
:103580001430B5EBC30F4FEAC30703D300200BB0D1
:10359000BDE8F08F2B199F42D8F80C303ABF7F1B43
:1035A000FFB227461BB9D8F81030002B7AD0272D50
:1035B0004ED8C5F12806B7424FF000032CBFF6B233
:1035C0003E4600932946D8F8080008AB3246FFF77C
:1035D00033FCA7EB060A35445FFA8AFAB8F81430D0
:1035E00003F10053053BDB000493D8F80C30039340
:1035F0002821039B13B1BAF1000F2CD1D8F8100089
:1036000040B1BAF1000F05D0009608AB5246691AD6
:10361000FFF712FC38B2002FB8D066070AD00AAB09
:1036200003EBD401624211F8083C02F00702134197
:1036300001F8083C082C3CD9102C40F2B580202C15
:1036400040F2B780BBF1000F00F09C80082334E00B
:10365000BA460026C2E7049BE02B28BFE02306936E
:103660000B44AB42059314D95A1B0398009692451C
:1036700034BF5246D2B2691A08AB04300792FFF742
:10368000DBFB079A1644AAEB020A1544F6B25FFA6E
:103690008AFA049B069A05999B1A0493039B1B685C
:1036A0000393A6E70093D8F8080008AB3A462946EA
:1036B000AEE7BBF1000F13D00123B4EBC30F6CD006
:1036C000082C12D89DF82030621E23FA02F2D5078A
:1036D00006D54FF0FF3202FA04F423438DF8203070
:1036E0009DF8203089F8003051E7102C12D8BDF831
:1036F0002030621E23FA02F2D10706D54FF0FF32C6
:1037000002FA04F42343ADF82030BDF82030A9F8C4
:1037100000303CE7202C0FD80899631E21FA03F3F0
:10372000DA0705D54FF0FF3202FA04F40C4308948F
:10373000089BC9F800302AE7402C2BD0DDE908654A
:10374000611EC4F12102A4F1210326FA01F105FA58
:1037500002F225FA03F311431943CB0712D50122D4
:10376000A4F12003C4F1200102FA03F322FA01F1CB
:10377000A240524243EA010363EB430332432B432B
:10378000CDE90823DDE90823C9E90023FFE66FF04E
:103790000100FCE66FF00800F9E6082CA0D9102C17
:1037A000B3D9202CEED8C3E7BBF1000FADD0022374
:1037B00083E7BBF1000FBBD004237EE730B5012ABD
:1037C000144638BF0124402C85B028BF4024002572
:1037D000012ACDE9025518D81B788DF80830630707
:1037E0000AD004AB03EBD405624215F8083C02F0A2
:1037F0000702934005F8083C009103462246002149
:1038000002A8FFF719FB05B030BD082AE4D9102A39
:1038100003D81B88ADF80830E1E7202A8DBFD3E933
:1038200000231B680293CDE90223D8E710B5CB68CB
:103830001BB98B600B618B8210BD04691A681C6018
:103840000361C38A013BC382CA60F0E703064CBF31
:10385000C0F3C0300220704708B50246FFF7F6FFFC
:10386000022806D15306C2F30F2001D100F0030055
:1038700008BDC2F30740FBE72DE9F04F93B0CDE957
:1038800003230A6804461046FFF7E0FF022814BF2E
:10389000C2F306260026002A0D46824680F2F781F2
:1038A00012F0C04940F0F381097B002900F0EF815C
:1038B000022803D02378B34240F0EC81C2F30463C2
:1038C0000693104602F07F030593FFF7C5FF059BA3
:1038D00029444FEA834848EA0A4848EA4668CE78CD
:1038E00000230022CDE90823F309834648EA0008B3
:1038F000029367D0059B009302466768534608A968
:103900002046B847002800F0C881276A4FB94146D1
:1039100004F10C00FFF7F4FA074690B96FF00200CB
:1039200054E03B6998450DD03F68002FF9D14146DE
:1039300004F10C00FFF7E4FA07460028EED0236AF2
:103940003B60276297F817C006F01F08CCF3840C81
:10395000ACEB08001FFA80FE0028B8BF0EF1200073
:10396000A8EB0C031FFA83FED7E90221B8BF00B20F
:10397000002B0793BEBF0EF120031BB2079352EA40
:10398000010338D0039BDFF824E39A1A049B4FF01D
:10399000000C63EB010196457CEB01032BD36B7BA1
:1039A00097F81AE0734519D1029B002B78D00128B3
:1039B00021DC7868F8B9DFF8F0C2944570EB0103B8
:1039C00016D337E0276A27B96FF00C0013B0BDE8B3
:1039D000F08F3B699845B5D03F68F4E7B248904214
:1039E0007CEB010301D30020F0E7029B002BFAD00F
:1039F000079B0F2B17DCFA7DB30002F0030203F0E4
:103A00007C031343FB7539462046FFF7F9FA6B7BBD
:103A1000BB76029B3BB9FB7DC3F38402013262F3A8
:103A20008603FB75D0E76A7BBB7E9A42DBD1029BA3
:103A3000002B35D0B309022B32D0039BBB60049B13
:103A4000FB60142200210DA8FDF7C6FE039B0A931C
:103A5000049B0B932B1D0C932B7BADF83EB0013BCD
:103A6000DBB2ADF83C30069B8DF84230059B8DF8FB
:103A7000433094F82C308DF840A083F001038DF88A
:103A800044308DF84180A3680AA920469847FB7D01
:103A9000C3F38403013303F01F039B02FB82A2E7FD
:103AA000FB7DC6F34012B2EBD31F40F0F980C3F3A5
:103AB0008403434540F0FC80029A2B7BB609002A20
:103AC00052D016F0010661D1032B40F2F480039B23
:103AD000BB60049BFB60FB8A66F30903FB822B7BC4
:103AE000AE1D033BDBB23246394604F10C00FFF752
:103AF00099FA00280CDA39462046FFF781FAFB7D57
:103B0000C3F38403013303F01F039B02FB8205E729
:103B1000DDE90884AB883B834FF6FF73C9F12000D1
:103B2000A9F1200228FA09F104FA00F0014324FA6D
:103B300002F211431846C9B2FFF7B6F909F10809B4
:103B4000B9F1400F0346E9D1B8822A7B033AD2B2D9
:103B50003146FFF7BBF9FB7DB882DA43C2F3C012EE
:103B600062F3C713FB753EE786B92E1D013BDBB23E
:103B70003246394604F10C00FFF754FA0028BADB4C
:103B80002A7BB88A013AD2B23146E2E7F98AC1F318
:103B90000901013B0429DAB25BD8281D002307F193
:103BA0001B069A4208D910F801CB06F801C0013172
:103BB00001330529DBB2F4D103990A9104990B91E1
:103BC000934207F11B010C9138BF043379680D91C2
:103BD00034BF55FA83F300230E93FB8AADF83EB051
:103BE000C3F309031A44069B8DF84230059B8DF8F8
:103BF000433094F82C30ADF83C2083F001038DF86D
:103C0000443000238DF840A08DF841807B602A7BF2
:103C1000B88A013A291DFFF759F93B8BB8828342D4
:103C200003D1A3680AA92046984720460AA9FFF7AE
:103C3000FDFDFB7DBA8AC3F38403013303F01F0348
:103C40009B02FB823B8B9A420CBF00206FF010005E
:103C5000BCE67B68002BAFD0052001E01C3033466A
:103C60001E68002EFAD1091A081D2E1D184401EBFA
:103C7000090CBCF11B0F5FFA89F39DD89A429BD9BE
:103C800016F8013B00F8013B09F10109EFE76FF07D
:103C900009009BE66FF00A0098E66FF00B0095E6CE
:103CA0006FF00D0092E600BF40420F0080841E00BE
:103CB0006FF00E008AE66FF00F0087E6EFF30983DE
:103CC00005494A6B22F001024A63683383F309888D
:103CD000002383F31188704700EF00E0302080F369
:103CE000118862B60C4B0D4AD96821F4E0610904D1
:103CF000090C0A43DA60D3F8FC20094942F08072CB
:103D0000C3F8FC200A6842F001020A602022DA7738
:103D100083F82200704700BF00ED00E00003FA05C1
:103D2000001000E010B5302383F311880E4B5B6860
:103D300013F4006314D0F1EE103AEFF30984683CF9
:103D40004FF08073E361094BDB6B236684F30988D2
:103D500000F08AFB10B1064BA36110BD054BFBE7D9
:103D600083F31188F9E700BF00ED00E000EF00E009
:103D70003F030008420300080268436811430160E2
:103D800003B1184770470000024AD36843F0C003EC
:103D9000D360704700100140024AD36843F0C0036B
:103DA000D36070470044004010B50A4C0A4A2046D0
:103DB000002100F0A9FA094B094AC4E99723094CEC
:103DC000094A0021204600F09FFA0849084BC4E93F
:103DD000971310BD704B0020893D000880F0FA0257
:103DE00000100140DC4D0020993D000800440040D7
:103DF00040787D012A4A037C002918BF0A46012B1E
:103E000030B5C0F868220CD1264B984239D1264BE8
:103E1000596C41F010015964596E41F01001596616
:103E20005B6EB2F904501468D0F86032D0F85C12BE
:103E3000002D03EB5403B3FBF4F3BEBF23F00705DF
:103E400003F0070343EA450394888B60D38843F06B
:103E500040030B61138943F001034B6144F40453A5
:103E600043F02C03CB6004F4A05400230B60B4F5A2
:103E7000806F0B684B680CBF7F23FF2380F8643290
:103E800030BD0A4B9842CCD1074B196C41F400313C
:103E90001964196E41F4003119661B6EC1E700BF49
:103EA000A0540008704B002000380240DC4D002078
:103EB0002DE9F041D0F85C62F7683368DA05044612
:103EC0009DB20DD5302383F311884FF48061043007
:103ED000FFF752FF6FF480733360002383F3118880
:103EE000302383F3118804F1040815F02F033AD12D
:103EF00083F31188380615D5290613D5302383F3AB
:103F0000118804F1380000F07BF900284EDA08210E
:103F1000201DFFF731FF4FF67F733B40F360002316
:103F200083F311887A0616D56B0614D5302383F3F4
:103F30001188D4E913239A420AD1236C43B127F0A4
:103F400040073F041021201D3F0CFFF715FFF760CD
:103F5000002383F31188D4F86822D36843B3BDE803
:103F6000F041106918472B0714D015F0080F0CBF4B
:103F700000214FF48071E80748BF41F02001AA07F3
:103F800048BF41F040016B0748BF41F08001404607
:103F9000FFF7F2FEAD06736805D594F8641220466B
:103FA000194000F0E1F93568ADB29EE77060B6E700
:103FB000BDE8F08100F1604303F561430901C9B236
:103FC00083F80013012200F01F039A4043099B006D
:103FD00003F1604303F56143C3F880211A60704721
:103FE000F8B5154682680669AA420B46816938BF52
:103FF0008568761AB54204460BD218462A46FDF764
:10400000D9FBA3692B44A361A3685B1BA36028466B
:10401000F8BD0CD918463246FDF7CCFBAF1BE16862
:104020003A463044FDF7C6FBE3683B44EBE71846ED
:104030002A46FDF7BFFBE368E5E70000836893428B
:10404000F7B51546044638BF8568D0E90460361ACE
:10405000B5420BD22A46FDF7ADFB63692B44636181
:10406000A36828465B1BA36003B0F0BD0DD93246A0
:104070000191FDF79FFB0199E068AF1B3A4631447F
:10408000FDF798FBE3683B44E9E72A46FDF792FB1E
:10409000E368E4E710B50A440024C361029B84602E
:1040A000C0E90000C0E90511C1600261036210BDF2
:1040B00008B5D0E90532934201D1826882B982689D
:1040C000013282605A1C42611970D0E904329A426E
:1040D00024BFC3684361002100F068FA002008BDD6
:1040E0004FF0FF30FBE7000070B5302304460E466A
:1040F00083F31188A568A5B1A368A269013BA360F9
:10410000531CA36115782269934224BFE368A3611D
:10411000E3690BB120469847002383F311882846B2
:1041200007E03146204600F031FA0028E2DA85F354
:10413000118870BD2DE9F74F04460E461746984684
:10414000D0F81C904FF0300A8AF311884FF0000B22
:10415000154665B12A4631462046FFF741FF034622
:1041600060B94146204600F011FA0028F1D0002342
:1041700083F31188781B03B0BDE8F08FB9F1000F0D
:1041800003D001902046C847019B8BF31188ED1A9C
:104190001E448AF31188DCE7C0E90511C160C361E0
:1041A0001144009B8260C0E9000001610362704716
:1041B000F8B504460D461646302383F31188A768E8
:1041C000A7B1A368013BA36063695A1C62611D70BB
:1041D000D4E904329A4224BFE3686361E3690BB116
:1041E00020469847002080F3118807E0314620469A
:1041F00000F0CCF90028E2DA87F31188F8BD00005E
:10420000D0E905239A4210B501D182687AB9826853
:10421000013282605A1C82611C7803699A4224BF71
:10422000C3688361002100F0C1F9204610BD4FF042
:10423000FF30FBE72DE9F74F04460E461746984638
:10424000D0F81C904FF0300A8AF311884FF0000B21
:10425000154665B12A4631462046FFF7EFFE034674
:1042600060B94146204600F091F90028F1D00023C2
:1042700083F31188781B03B0BDE8F08FB9F1000F0C
:1042800003D001902046C847019B8BF31188ED1A9B
:104290001E448AF31188DCE7026843681143016019
:1042A00003B11847704700001430FFF743BF000008
:1042B0004FF0FF331430FFF73DBF00003830FFF7F9
:1042C000B9BF00004FF0FF333830FFF7B3BF000035
:1042D0001430FFF709BF00004FF0FF311430FFF733
:1042E00003BF00003830FFF763BF00004FF0FF321C
:1042F0003830FFF75DBF0000012914BF6FF01300D5
:1043000000207047FFF750BD37B515460E4A0260D2
:1043100000224260C0E902220122044602740B46D8
:10432000009000F15C014FF480721430FFF7B2FE90
:1043300000942B464FF4807204F5AE7104F13800FE
:10434000FFF72AFF03B030BDB454000810B5302386
:10435000044683F31188FFF74DFD022323740020E8
:1043600080F3118810BD000038B5C36904460D46BE
:104370001BB904210844FFF78FFF294604F11400FC
:10438000FFF796FE002806DA201D4FF40061BDE815
:104390003840FFF781BF38BD002303758268036989
:1043A0001B6899689142FBD25A68036042601060B2
:1043B0005860704700230375826803691B68996819
:1043C0009142FBD85A6803604260106058607047A1
:1043D00008B50846302383F311880B7D032B05D0E5
:1043E000042B0DD02BB983F3118808BD8B690022F3
:1043F0001A604FF0FF338361FFF7CEFF0023F2E72F
:10440000D1E9003213605A60F3E70000FFF7C4BF40
:10441000054BD9680875186802681A605360012254
:104420000275D860FBF776BF4850002030B50C4BC2
:10443000DD684B1C87B004460FD02B46094A6846FE
:1044400000F046F92046FFF7E3FF009B13B16846F2
:1044500000F048F9A86907B030BDFFF7D9FFF9E7C8
:1044600048500020D1430008044B1A68DB6890686C
:104470009B68984294BF002001207047485000205C
:10448000084B10B51C68D86822681A605360012276
:104490002275DC60FFF78EFF01462046BDE8104024
:1044A000FBF738BF4850002038B5074C074908488B
:1044B000012300252370656000F028FC022323708F
:1044C00085F3118838BD00BFB0520020E0540008C9
:1044D0004850002008B572B6044B186500F0E0FAA9
:1044E00000F088FB024B03221A70FEE748500020C0
:1044F000B052002000F02CB98B60022308618B823F
:10450000084670478368A3F1840243F8142C0269BB
:1045100043F8442C426943F8402C094A43F8242CC0
:10452000C26843F8182C022203F80C2C002203F86E
:104530000B2C044A43F8102CA3F12000704700BF55
:104540002D0300084850002008B5FFF7DBFFBDE849
:104550000840FFF75BBF0000024BDB6898610F204B
:10456000FFF756BF48500020302383F31188FFF730
:10457000F3BF000008B50146302383F311880820FB
:10458000FFF754FF002383F3118808BD064BDB6857
:1045900039B1426818605A60136043600420FFF725
:1045A00045BF4FF0FF3070474850002003689842E5
:1045B00006D01A680260506099611846FFF726BF5E
:1045C0007047000010B503689C68A2420CD85C6874
:1045D0008A600B604C602160596099688A1A9A6001
:1045E0004FF0FF33836010BD1B68121BECE7000027
:1045F0000A2938BF0A2170B504460D460A266019FB
:1046000000F07CFB00F064FB041BA54203D8751C82
:104610002E460446F3E70A2E04D9BDE87040012077
:1046200000F0B4BB70BD0000F8B5144B0D46D96165
:1046300003F1100141600A2A1969826038BF0A2219
:10464000016048601861A818144600F047FB0A276B
:1046500000F03EFB431BA342064606D37C1C2819F0
:1046600000F04CFB27463546F2E70A2F04D9BDE897
:10467000F840012000F08ABBF8BD00BF4850002080
:10468000F8B506460D4600F023FB0F4A134653F8D3
:10469000107F9F4206D12A4601463046BDE8F840C9
:1046A000FFF7C2BFD169BB68441A2C1928BF2C463A
:1046B000A34202D92946FFF79BFF22463146034811
:1046C000BDE8F840FFF77EBF48500020585000205A
:1046D00010B4C0E9032300235DF8044B4361FFF7E6
:1046E000CFBF000010B5194C236998420DD0D0E916
:1046F0000032816813605A609A680A449A60002305
:1047000003604FF0FF33A36110BD2346026843F8F6
:10471000102F53600022026022699A4203D1BDE843
:10472000104000F0E5BA936881680B44936000F094
:10473000CFFA2269E1699268441AA242E4D911448D
:10474000BDE81040091AFFF753BF00BF48500020D2
:104750002DE9F047DFF8BC8008F110072C4ED8F89F
:10476000105000F0B5FAD8F81C40AA68031B9A4212
:104770003ED81444D5E900324FF00009C8F81C4077
:1047800013605A60C5F80090D8F81030B34201D1D8
:1047900000F0AEFA89F31188D5E90331284698472D
:1047A000302383F311886B69002BD8D000F090FA86
:1047B0006A69A0EB04094A4582460DD2022000F046
:1047C000E5FA0022D8F81030B34208D15146284605
:1047D000BDE8F047FFF728BF121A2244F2E712EBB8
:1047E000090938BF4A4629463846FFF7EBFEB5E7C8
:1047F000D8F81030B34208D01444211AC8F81C006D
:10480000A960BDE8F047FFF7F3BEBDE8F08700BF41
:10481000585000204850002038B500F059FA054A99
:10482000D2E90845031B181945F10001C2E9080146
:1048300038BD00BF4850002000207047FEE7000050
:10484000704700004FF0FF3070470000BFF34F8FFC
:10485000024AD368DB03FCD4704700BF003C02402F
:1048600008B5094B1B7873B9FFF7F0FF074B1A69BE
:10487000002ABFBF064A5A6002F188325A601A689D
:1048800022F480621A6008BDB8520020003C024049
:104890002301674508B50B4B1B7893B9FFF7D6FF8B
:1048A000094B1A6942F000421A611A6842F48052B8
:1048B0001A601A6822F480521A601A6842F4806200
:1048C0001A6008BDB8520020003C02400B28F0B529
:1048D00016D80C4C0C4923787BB90C4D0E460C2392
:1048E0004FF0006255F8047B46F8042B013B13F0AF
:1048F000FF033A44F6D10123237051F82000F0BDA4
:104900000020FCE7EC520020BC520020EC540008D0
:10491000014B53F820007047EC5400080C207047FE
:104920000B2810B5044601D9002010BDFFF7CEFFBB
:10493000064B53F824301844C21A0BB90120F4E78F
:1049400012680132F0D1043BF6E700BFEC540008D6
:104950000B2810B5044621D8FFF778FFFFF780FF3A
:104960000F4AF323D360C300DBB243F4007343F078
:1049700002031361136943F480331361FFF766FF89
:10498000FFF7A4FF074B53F8241000F02FF9FFF7AF
:1049900081FF2046BDE81040FFF7C2BF002010BDD8
:1049A000003C0240EC540008F8B512F00103144634
:1049B00042D18218B2F1016F57D82D4B1B6813F00A
:1049C000010352D02B4DFFF74BFFF323EB60FFF7B2
:1049D0003DFF40F20127032C15D824F0010466188E
:1049E000244C401A40F20117B142236900EB010543
:1049F00024D123F001032361FFF74CFF0120F8BD10
:104A0000043C0430E7E78307E7D12B6923F44073C4
:104A10002B612B693B432B6151F8046B0660BFF39C
:104A20004F8FFFF713FF03689E42E9D02B6923F0F5
:104A300001032B61FFF72EFF0020E0E723F4407312
:104A4000236123693B4323610B882B80BFF34F8F86
:104A5000FFF7FCFE2D8831F8023BADB2AB42C3D06C
:104A6000236923F001032361E4E71846C7E700BF89
:104A700000380240003C0240084908B50B7828B1D4
:104A80001BB9FFF7EDFE01230B7008BD002BFCD016
:104A9000BDE808400870FFF7FDBE00BFB852002017
:104AA0000149024800F0A4B800FF03000001002003
:104AB0000846114600F01EBC084600F031BC00005C
:104AC00038B5EFF311859DB9EFF30584C4F30804FD
:104AD000302334B183F31188FFF79EFE85F31188EC
:104AE00038BD83F31188FFF797FE84F3118838BD32
:104AF000BDE83840FFF790BE38B5FFF7E1FF114C35
:104B0000114AC00840EA4170A0FB025EC908A0FB40
:104B1000040C1CEB050CA1FB04404FF000035B41AF
:104B2000A1FB02121CEB040C43EB000011EB0E0185
:104B300042F10002411842F10000090941EA007007
:104B400038BD00BFCFF753E3A59BC42010B5024486
:104B5000064BD2B2904200D110BD441C00B253F8B3
:104B6000200041F8040BE0B2F4E700BF50280040F9
:104B70000F4B30B51C6F240407D41C6F44F4007431
:104B80001C671C6F44F400441C670A4C236843F400
:104B9000807323600244084BD2B2904200D130BDF2
:104BA000441C00B251F8045B43F82050E0B2F4E733
:104BB00000380240007000405028004007B5012234
:104BC00001A90020FFF7C2FF019803B05DF804FBC4
:104BD00013B50446FFF7F2FFA04205D0012201A958
:104BE00000200194FFF7C4FF02B010BD7047000021
:104BF0007047000070470000074B45F255521A609D
:104C000003225A6040F2FF729A604CF6CC421A605E
:104C1000024B01221A70704700300040F45200200D
:104C2000034B1B781BB1034B4AF6AA221A6070474C
:104C3000F452002000300040034B1A681AB9034AAE
:104C4000D2F874281A607047F052002000300240F9
:104C5000024B4FF08072C3F8742870470030024056
:104C600008B5FFF7E9FF024B1868C0F3407008BDB4
:104C7000F052002008B5FFF7DFFF024B1868C0F3C1
:104C8000007008BDF052002070470000FEE70000F1
:104C90000A4B0B480B4A90420BD30B4BDA1C121AEF
:104CA000C11E22F003028B4238BF00220021FCF714
:104CB00093BD53F8041B40F8041BECE7945600081E
:104CC00078530020785300207853002000F0D0B8AB
:104CD000014B586A704700BF000C0040034B002294
:104CE00058631A610222DA60704700BF000C00406E
:104CF000014B0022DA607047000C0040014B586302
:104D0000704700BF000C0040FEE7000070B51B4B71
:104D100001630025044686B0586085620E46FEF7A2
:104D2000DDFF04F11003C4E904334FF0FF33C4E99D
:104D30000635C4E90044A560E562FFF7C9FF2B46CC
:104D40000246C4E9082304F134010D4A2565802395
:104D50002046FFF7D1FB0123E0600A4A0375009269
:104D600072680192B268CDE90223074B6846CDE92B
:104D70000435FFF7E9FB06B070BD00BFB05200205C
:104D80001C55000821550008094D0008024AD36A45
:104D90001843D062704700BF485000204B68436002
:104DA0008B688360CB68C3600B6943614B690362A6
:104DB0008B6943620B6803607047000008B5234BA2
:104DC00023481A6942F0FF021A611A6922F0FF02B1
:104DD0001A611A691A6B42F0FF021A631A6D42F0E7
:104DE000FF021A651B4A1B6D1146FFF7D7FF02F140
:104DF0001C0100F58060FFF7D1FF02F1380100F5DA
:104E00008060FFF7CBFF02F1540100F58060FFF7EF
:104E1000C5FF02F1700100F58060FFF7BFFF02F1EE
:104E20008C0100F58060FFF7B9FF02F1A80100F5E1
:104E30008060FFF7B3FF02F1C40100F58060FFF767
:104E4000ADFFBDE8084000F08FB800BF0038024059
:104E5000000002402855000808B500F029FAFFF7C5
:104E600023FBBDE80840FFF7E7BE000070470000E5
:104E70000E4B1A6C42F008021A641A6E42F00802D5
:104E80001A660B4A1B6E936843F008039360094B44
:104E900031229A624FF0FF32DA6200229A615A633D
:104EA000DA605A6001225A611A6070470038024085
:104EB000002004E0000C0040094A08B51169D368DD
:104EC0000B40D9B2C9439B07116107D5302383F347
:104ED0001188FFF70FFB002383F3118808BD00BF83
:104EE000000C00401E4B1A6962F0FF021A611A6939
:104EF000D2B21A614FF0FF301A695A695861002125
:104F00005A6959615A691A6A62F080521A621A6AB9
:104F100002F080521A621A6A5A6A58625A6A5962D0
:104F20005A6A1A6C42F080521A641A6E42F0805229
:104F30001A661A6E0B4A106840F480701060186F81
:104F400000F44070B0F5007F1EBF4FF4803018674A
:104F50001967536823F40073536000F07DB900BFF4
:104F600000380240007000403B4B3C4A1A643C4A07
:104F70004FF4404111601A6842F001021A601A6849
:104F80009007FCD59A6822F003029A60324B9A6827
:104F900012F00C02FBD1196801F0F90119609A6056
:104FA0001A6842F480321A601A689103FCD55A6F6D
:104FB00042F001025A67284B5A6F9207FCD5294AE2
:104FC0005A601A6842F080721A60254A5368580481
:104FD000FCD5214B1A689101FCD5234AC3F88420E3
:104FE0001A6842F080621A601A681201FCD51F4AE2
:104FF0009A600322C3F88C204FF00062C3F894201B
:105000001B4B1A681B4B9A421B4B21D11B4A116840
:105010001B4A91421CD140F203121A60164A1368CF
:1050200003F00F03032BFAD10B4B9A6842F00202F4
:105030009A609A6802F00C02082AFAD15A6C42F47B
:1050400080425A645A6E42F480425A665B6E7047E0
:1050500040F20372E1E700BF003802400004001094
:105060000070004004194002083000240094883881
:10507000002004E011640020003C024000ED00E04C
:1050800041C20F41074A08B5536903F00103536158
:1050900023B1054A13680BB150689847BDE8084032
:1050A000FEF740BE003C0140F8520020074A08B518
:1050B000536903F00203536123B1054A93680BB1AE
:1050C000D0689847BDE80840FEF72CBE003C014080
:1050D000F8520020074A08B5536903F004035361EE
:1050E00023B1054A13690BB150699847BDE80840E0
:1050F000FEF718BE003C0140F8520020074A08B5F0
:10510000536903F00803536123B1054A93690BB156
:10511000D0699847BDE80840FEF704BE003C014056
:10512000F8520020074A08B5536903F01003536191
:1051300023B1054A136A0BB1506A9847BDE808408D
:10514000FEF7F0BD003C0140F8520020164B10B5B0
:105150005C6904F478725A61A30604D5134A936A11
:105160000BB1D06A9847600604D5104A136B0BB197
:10517000506B9847210604D50C4A936B0BB1D06B4A
:105180009847E20504D5094A136C0BB1506C984757
:10519000A30504D5054A936C0BB1D06C9847BDE8C4
:1051A0001040FEF7BFBD00BF003C0140F852002098
:1051B000194B10B55C6904F47C425A61620504D550
:1051C000164A136D0BB1506D9847230504D5134A49
:1051D000936D0BB1D06D9847E00404D50F4A136E60
:1051E0000BB1506E9847A10404D50C4A936E0BB1D5
:1051F000D06E9847620404D5084A136F0BB1506F04
:105200009847230404D5054A936F0BB1D06F984794
:10521000BDE81040FEF786BD003C0140F85200207A
:1052200008B50348FEF744FEBDE80840FEF77ABD26
:10523000704B002008B50348FEF73AFEBDE8084071
:10524000FEF770BDDC4D002008B5FFF735FEBDE868
:105250000840FEF767BD0000062108B50846FEF7C6
:10526000A9FE06210720FEF7A5FE06210820FEF76D
:10527000A1FE06210920FEF79DFE06210A20FEF769
:1052800099FE06211720FEF795FE06212820FEF73D
:1052900091FE07213220FEF78DFE0C212520FEF71E
:1052A00089FEBDE808400C212620FEF783BE0000E1
:1052B00008B5FFF717FE00F009F8FFF723F8FFF72E
:1052C000D5FDBDE80840FFF701BD00000023054AF9
:1052D00019460133102BC2E9001102F10802F8D17E
:1052E000704700BFF85200200B460146184600F0F8
:1052F00009B80000024B0A4601461868FFF7D8BB00
:105300002823002010B5054C13462CB10A4601464F
:105310000220AFF3008010BD2046FCE70000000033
:10532000024B01461868FFF7C7BB00BF28230020C7
:1053300010B501390244904201D1002005E0037804
:1053400011F8014FA34201D0181B10BD0130F2E744
:105350002DE9F041A3B1C91A17780144044603F1BD
:10536000FF3C8C42204601D9002009E00578BD426F
:1053700004F10104F5D10CEB0405D618A54201D1C6
:10538000BDE8F08115F8018D16F801EDF045F5D076
:10539000E7E70000034611F8012B03F8012B002A70
:1053A000F9D170476F72672E6172647570696C6FA6
:1053B000742E41524B5F43414E4E4F444500000016
:1053C00053544D3332463F3F3F0053544D333246E2
:1053D0003430780053544D333246343278005354CD
:1053E0004D33324634343658580000000120330023
:1053F0000010410001105A0003105900071031003D
:1054000000000000C053000813040000CA53000845
:1054100019040000D453000821040000DE530008E2
:1054200040A2E4F1646891060041A3E5F265699247
:10543000070000004261642043414E496661636594
:1054400020696E6465782E008000000000800000F6
:105450000000800000000000000000002121000882
:1054600065290008C1280008612100086D21000895
:105470007923000831210008412100083521000866
:105480003D21000839210008952200084521000827
:10549000892C0008392C00085521000869220008D1
:1054A0000096000000000000000000000000000066
:1054B0000000000000000000C5420008B1420008E2
:1054C000ED420008D9420008E5420008D142000838
:1054D000BD420008A9420008F942000863300000FC
:1054E000DC540008A0500020B05200200040000012
:1054F00000400000004000000040000000000100EB
:105500000000020000000200000002000000020093
:105510000000020000000200000002006D61696EE0
:105520000069646C65000000A00195AA00070000F6
:10553000AAAAAAAA50010064FFF90000007700009F
:10554000009009708000000100000000AAAAAAAA29
:1055500040000001FFFF000000700000000000009C
:105560000000005000000000AAAAAA5A0000000093
:10557000FF3F0000000000000000000000000000ED
:1055800000000000AAAAAAAA00000000FFFF000075
:10559000000000000000000000000000000000000B
:1055A000AAAAAAAA00000000FFFF00000000000055
:1055B000000000000000000000000000AAAAAAAA43
:1055C00000000000FFFF00000000000000000000DD
:1055D0000000000000000000AAAAAAAA0000000023
:1055E000FFFF0000000000000000000000000000BD
:1055F000000000000A00000000000000030000009E
:105600000000000000000000530000000000000047
:1056100000000F000000000040420F00FE2A0100C1
:10562000D2040000FF000000704B0020DC4D002081
:105630002C230020000000000000000000000000FB
:10564000000000000000000000000000000000005A
:10565000000000000000000000000000000000004A
:10566000000000000000000000000000000000003A
:10567000000000000000000000000000000000002A
:10568000000000000000000000000000000000001A
:045690000000000016
:00000001FF
